:060000000A128A11122809
:10000800FE00030EFA000408FB000A08FC00831235
:1000180003137F08FD000A128A15612F0A128A113C
:1000280015288313203084003B300A128A15E426F1
:1000380083010A128A1120280730831603139F00B0
:10004800C03081000B17831203131210921012157F
:100058001208073948389200F930831603139200C2
:100068008B178C14FE3083120313D00050088316AC
:100078000313850583120508FE398500FD30D0007D
:10008800500883160313850583120508FD3985007A
:10009800FB30D0005008831603138505831205082A
:1000A800FB398500F730D000500883160313850507
:1000B80083120508F7398500EF30D0005008831601
:1000C8000313870583120708EF398700F730D0003C
:1000D800500883160313870583120708F73987002A
:1000E800FD30D000500883160313870583120313CD
:1000F80007080238870001300A128A15D9270A1220
:100108008A11831203133803031D052AFE30D00019
:100118005008831603138505831203130508013855
:100128008500FD30D000500883160313850583121F
:100138000313050802388500FB30D00050088316E9
:100148000313850583120313050804388500F73067
:10015800D00050088316031385058312031305087E
:1001680008388500FE30D000500883160313870531
:10017800831203130708013887000130D0005008A4
:10018800B2000A128A15FA260A128A110A128A1568
:1001980049270A128A1183120313D0005008AD00B0
:1001A800F730D00050088316031387058312031312
:1001B800070808388700FE30D0005008831603135C
:1001C800850583120508FE39850032300A128A1522
:1001D80033270A128A11F73083120313D00050080C
:1001E80083160313870583120708F73987000A1255
:1001F8008A11F1270A128A110A128A15FA260A1296
:100208008A110A128A1549270A128A1183120313BE
:10021800D0005008AF00F730D00050088316031301
:10022800870583120313070808388700FD30D000BC
:10023800500883160313850583120508FD398500C8
:1002480032300A128A1533270A128A11F7308312BC
:100258000313D00050088316031387058312070879
:10026800F73987000A128A11F1270A128A110A122D
:100278008A15FA260A128A110A128A1549270A12B9
:100288008A1183120313D0005008B000F730D00051
:1002980050088316031387058312031307080838C9
:1002A8008700FB30D000500883160313850583129E
:1002B8000508FB39850032300A128A1533270A12DD
:1002C8008A11F73083120313D000500883160313E2
:1002D800870583120708F73987000A128A11F12760
:1002E8000A128A110A128A15FA260A128A110A12A1
:1002F8008A1549270A128A1183120313D00050085D
:10030800B100F730D0005008831603138705831215
:100318000313070808388700F730D0005008831601
:100328000313850583120508F739850032300A1250
:100338008A1533270A128A11F73083120313D00063
:10034800500883160313870583120708F7398700B7
:100358000A128A11F1270A128A1100308312031334
:10036800C000C1002D08D000D1015008C2005108BA
:10037800C3000A128A15EC260A128A110130831268
:100388000313C0000030C1002F08D000D10150086D
:10039800C2005108C3000A128A15EC260A128A11F3
:1003A800023083120313C0000030C1003008D000AF
:1003B800D1015008C2005108C3000A128A15EC2660
:1003C8000A128A11033083120313C0000030C100DF
:1003D8003108D000D1015008C2005108C3000A12E8
:1003E8008A15EC260A128A1183120313B201FE3011
:1003F800D000500883160313870583120708FE39B7
:1004080087000030C100C2000A128A151F270A128D
:100418008A11831203134108D0005008AD0001303F
:10042800C1000030C2000A128A151F270A128A1159
:10043800831203134108D0005008AF000230C100F6
:100448000030C2000A128A151F270A128A11831265
:1004580003134108D0005008B0000330C100003039
:10046800C2000A128A151F270A128A11831203135F
:100478004108D0005008B10014300A128A153327F9
:100488000A128A110A128A15FA260A128A110A12FF
:100498008A1549270A128A1183120313D0005008BB
:1004A800B600360A03198F2A0A30360603198F2A2E
:1004B8003308031D8F2A3408013ED0005008B400C9
:1004C8000130D0005008B300A601A701A801A90176
:1004D800AC01B5010330390603198F2AF730D00073
:1004E8005008831603138705831203130708083877
:1004F800870032300A128A1533270A128A11F73018
:1005080083120313D0005008831603138705831240
:100518000708F73987000A303606031D8A2BFE3094
:10052800D000500883160313850583120508FE3989
:100538008500FD30D000500883160313850583120B
:100548000508FD398500FB30D000500883160313D9
:10055800850583120508FB398500F730D00050085F
:1005680083160313850583120508F7398500EF30D4
:10057800D000500883160313870583120708EF3944
:100588008700B901B401F730D0005008831603136F
:1005980087058312031307080838870032300A12C8
:1005A8008A1533270A128A11F73083120313D000F1
:1005B800500883160313870583120708F739870045
:1005C8008A2BFE30D000500883160313850583124A
:1005D800031305080138882BFD30D0005008831616
:1005E800031385058312031305080238882BFB3093
:1005F800D0005008831603138505831203130508DA
:100608000438882B0330390603192C2DF730D00015
:100618005008831603138505831203130508083849
:100628008500F730D000500883160313870583121E
:1006380003130708083887002E08013ED000500829
:10064800AE0001300A128A15D9270A128A11FE3023
:1006580083120313D00050088316031385058312F1
:100668000508FE398500FD30D000500883160313B5
:10067800850583120508FD398500FB30D000500838
:1006880083160313850583120508FB398500F730A7
:10069800D000500883160313850583120508F7391F
:1006A8008500B401F730D00050088316031387057E
:1006B80083120708F73987002C2DFE30D000500828
:1006C80083160313850583120508FE398500FD305E
:1006D800D000500883160313850583120508FD39D9
:1006E8008500FB30D000500883160313850583125C
:1006F8000508FB398500F730D0005008831603132E
:10070800850583120508F73985002C2D3408013A30
:100718000319E52A033A0319F02A013A0319FB2AB7
:10072800073A0319062B612B2C2D36082F06031DBB
:100738001E2D0230A42B36083006031D1E2D033053
:10074800D0005008B9001E2D36083106031DB92CFB
:10075800F730D0005008831603138505831203135E
:10076800050808388500BA0105303A0203183D2CFF
:10077800F730D0005008831603138705831203133C
:10078800070808388700FE30D00050088316031386
:10079800850583120313050801388500FD30D00054
:1007A80050088316031385058312031305080238BE
:1007B8008500FB30D000500883160313850583128B
:1007C8000313050804388500F730D0005008831655
:1007D8000313850583120313050808388500323092
:1007E8000A128A1533270A128A11F7308312031363
:1007F800D000500883160313870583120708F739BA
:100808008700FE30D0005008831603138505831235
:100818000508FE398500FD30D00050088316031303
:10082800850583120508FD398500FB30D000500886
:1008380083160313850583120508FB398500F730F5
:10084800D000500883160313850583120508F7396D
:10085800850032300A128A1533270A128A110130AC
:1008680083120313D0005008BA0705303A02031C5C
:10087800BC2BEF30D0005008831603138705831272
:100888000313070810388700FB30D0005008831680
:100898000313870583120313070804388700FD3004
:1008A800D000500883160313870583120708FD3903
:1008B8008700AE01BF30D0005008831603138705A8
:1008C80083120708BF39870002300A128A15D92710
:1008D8000A128A11FE3083120313D00050088316BF
:1008E8000313850583120508FE398500FD30D00005
:1008F800500883160313850583120508FD39850002
:10090800FB30D000500883160313850583120508B1
:10091800FB398500F730D00050088316031385058E
:1009280083120508F7398500EF30D0005008831688
:100938000313870583120708EF398700FB30D000BF
:10094800500883160313870583120708FB398700AD
:10095800FD30D00050088316031387058312031354
:10096800070802388700B901B401360831060319AF
:100978001E2DF730D0005008831603138505831207
:100988000313050808388500F730D000500883168F
:1009980003138705831203130708083887002E08F6
:1009A800013ED0005008AE0001300A128A15D9273E
:1009B8000A128A11FE3083120313D00050088316DE
:1009C8000313850583120508FE398500FD30D00024
:1009D800500883160313850583120508FD39850021
:1009E800FB30D000500883160313850583120508D1
:1009F800FB398500F730D0005008831603138505AE
:100A080083120508F7398500F730D000500883169F
:100A18000313870583120708F7398700EF30D000E2
:100A2800500883160313870583120708EF398700D8
:100A3800B901B4013408031D372DB901372D360823
:100A48002D06031D372D0130D0005008B900372D71
:100A58003908013A0319992B033A03199F2B013AD4
:100A68000319A82B232D0A128A11F1270A128A11B9
:100A78000330831203132E02031C512DBF30D00004
:100A88005008831603138705831203130708403899
:100A980087000330D0005008AE00B301402A532D20
:100AA80083120313CC010A128A11F9250A128A113A
:100AB80083120313CC01FF30C8004808CA00F32D85
:100AC800FE30C800480883160313860583120313F3
:100AD80006080138842DFD30C80048088316031322
:100AE80086058312031306080238842DFB30C800DC
:100AF800480883160313860583120313060804386F
:100B08008600942D4C08003A0319642D013A031904
:100B18006F2D033A03197A2D013A0319942D942D58
:100B280014300A128A1196270A128A110A128A1197
:100B380026270A128A1183120313C8004808CB001B
:100B4800C42DFE30C8004808831603138605831297
:100B58000608FE39C22DFD30C80048088316031365
:100B6800860583120608FD39C22DFB30C8004808E7
:100B780083160313860583120608FB398600D22DD7
:100B88004C08003A0319A52D013A0319AF2D033A71
:100B98000319B92D013A0319D22DD22D4B0A031985
:100BA800E62D0330C8004808BB004B080A128A1516
:100BB8000C270A128A11831203134C07C90049082B
:100BC800CA00F72D32300A128A1196270A128A11A2
:100BD800831203134C08013EC8004808CC000330B8
:100BE8004C02031C862D4A08080083120313C60111
:100BF800462E0630BB000030BC008630BD000030F9
:100C0800BE001030C2004208BF000430342E063047
:100C1800BB000030BC008630BD000030BE00203074
:100C2800C2004208BF000530342E0630BB00003039
:100C3800BC008630BD000030BE004030C200420813
:100C4800BF000630342E0630BB000030BC008630B2
:100C5800BD000030BE008030C2004208BF0007302F
:100C6800C3004308C0000A128A15B7270A128A115E
:100C780083120313C4004408C5004608013EC2009D
:100C88004208C600043046020318592E4608003AA6
:100C98000319FD2D013A03190B2E033A0319192ED6
:100CA800013A0319272E412E412EC6017E2EFE3011
:100CB800C200420883160313860583120608FE390C
:100CC800782EFD30C200420883160313860583126E
:100CD8000608FD39782EFB30C2004208831603133C
:100CE800860583120608FB3986004608013EC200C5
:100CF8004208C60003304602031808004608003AB6
:100D080003195B2E013A0319652E033A03196F2E56
:100D1800013A0319792E792E792E0730F000003028
:100D2800F1008730F2000030F3002030F700770838
:100D3800F4000530F8007808F5000A128A1597279C
:100D48000A128A11F900790883120313B8003203D2
:100D5800031908002608013EA60027080318013ECB
:100D6800003EA7002808013EA80029080318013EF4
:100D7800003EA900D0302606073003192706031DB8
:100D8800072FA601A7013508013EF7007708B5002F
:100D980005303506031D072FFE30F7007708831648
:100DA8000313850583120508FE398500FD30F70019
:100DB800770883160313850583120508FD39850016
:100DC800FB30F7007708831603138505831205089F
:100DD800FB398500F730F70077088316031385057C
:100DE80083120508F7398500B501A601A701EF3080
:100DF800F700770883160313870583120708EF396E
:100E08008700B901B401D030280607300319290634
:100E1800031D0800A801A9012C08013EF700770866
:100E2800AC003D302C02031C0800AC01AE01BF3001
:100E3800F700770883160313870583120708BF395D
:100E48008700080083120313C701C601C701FF30DA
:100E5800C2004208C500902F0630BB000030BC001D
:100E68008630BD000030BE001030C2004208BF000E
:100E78000430672F0630BB000030BC008630BD0050
:100E88000030BE002030C2004208BF000530672F86
:100E98000630BB000030BC008630BD000030BE000C
:100EA8004030C2004208BF000630672F0630BB0042
:100EB8000030BC008630BD000030BE008030C2006B
:100EC8004208BF000730C3004308C0000A128A1551
:100ED800B7270A128A1183120313C4004408C600F4
:100EE800832F4708003A0319302F013A03193E2F80
:100EF800033A03194C2F013A03195A2F832F460836
:100F080003198B2F4708C2004208C500942F4708D1
:100F1800013EC2004208C70004304702031C752F77
:100F28004508080083120313BC0064303C02031C0C
:100F3800B42FA53083120313BB00BB0BA12FA42F22
:100F4800643083120313BC02992F0F3083120313EA
:100F5800BB00BB0BAD2FB02F0A3083120313BC02AA
:100F68000A303C02031CBC2FA92FBA2FBB2F00004C
:100F7800013083120313BC023C0A03190800B92F7D
:100F8800831603178C18C42F831203133B0883128C
:100F980003178D00831203133D08831203178C0077
:100FA800831603178C130C1500308B1B013083122A
:100FB8000313BF008B135530831603178D00AA3017
:100FC8008D008C148C18E62F831203133F08031D21
:100FD8008B17831603170C1108000A128A1154255F
:100FE8000A128A1183120313CD004D08CE004E0A4F
:060FF80003190800F12FAF
:1010000008308A000408840A82070034013402345C
:1010100003340434053406340734083409340A34FC
:1010200000340B34313432343334343435343634E0
:0E1030003734383439342A3430342334003421
:101DC80064008001840A0406031900340406E52E21
:101DD800831203134108BC004008BB004308BE003F
:101DE8004208BD000A128A11C42708000A128A1183
:101DF80054250A128A1583120313CD004D08CF000B
:101E08004F0A0319FA2E4F08CD004D08CE000800DE
:101E180083120313BE00BD013E1C162F3B08BC00F5
:101E28003C08BD070310BB0D0310BE0C3E08031D84
:101E3800102F3D080800831203134208BC00410814
:101E4800BB000A128A157B27831203133C08C400BF
:101E58003B08C3004408C2004308C10008008312BD
:101E68000313BD00013083120313BD023D0A031999
:101E78000800073083120313BC007C30BB00BB0B87
:101E8800432FBC0B432F0000362F0A128A1154250A
:101E98000A128A1583120313CD004D08CE004E0A8C
:101EA80003195F2F4E08013E84000A128A1500208C
:101EB800CD004D08CE004E0808008C1C6F2F8316ED
:101EC80003138C1C6F2F0A128A1191260A128A1585
:101ED800831203138C107D088312FF007C088A008C
:101EE8007B0884007A0E8300FE0E7E0E09008312A2
:101EF8000313BF01C0013B08831203178D0083162B
:101F080003178C130C14831203170C088312031382
:101F1800BD00BE013D08BF003E08C0004008BC002F
:101F28003F08BB000800720884008317731C8313E2
:101F380000087404F600720884008317731C831366
:101F480076088000700884008317711C83130008CA
:101F58007405F600750AB22F0310F60CFF3E031D38
:101F6800B02F76080800831203133D0884008317F6
:101F78003E1C831300083F04C1003D0884008317FA
:101F88003E1C8313410880003B08840083173C1CD7
:101F9800831300083F05C100400AD42F0310C10C69
:101FA800FF3E031DD22F4108080083120313BF0010
:101FB800C0013F08400203180800FA300A128A15C7
:101FC80033270A128A15FA300A128A1533270A1299
:101FD8008A15FA300A128A1533270A128A15FA3036
:101FE8000A128A1533270A128A150130831203133D
:081FF800BE003E08C007DD2F0A
:02400E0032FF7F
:104200000000010002000300410062004800650058
:104210006C006C006F00FF00FF00FF00FF00FF005C
:00000001FF
